:1000000012C02CC02BC02AC029C028C027C026C0BF
:1000100025C024C023C022C021C020C01FC01EC0D4
:100020001DC0A1C01BC011241FBECFE5D4E0DEBFA0
:10003000CDBF10E0A0E6B0E0EEE4F2E002C0059033
:100040000D92AE36B107D9F710E0AEE6B0E001C0D0
:100050001D92A037B107E1F702D0F7C0D1CFCF93FF
:10006000DF9314BE88E10FB6F89481BD11BC0FBEBA
:1000700086E087BB8CE084BB11BA82E4C8D032D062
:1000800041D078942DE088E190E00FB6F894A895DF
:1000900081BD0FBE21BD80E690E0C2D0D4E0C2E0B9
:1000A000CDD0882329F088B38D2788BB33D0B8D032
:1000B00088B38C2788BBA895F3CF97B1907F97B969
:1000C00097B18F70892B87B9369A089581E0369958
:1000D00080E00895FBDF8823E9F3369824B135B139
:1000E000C901089517B83E9A86B1856086B9379AD6
:1000F00080E0E3DFEFDF0895EDDF96958795969535
:1001000087950895AB9AAA98089581E0D6DFF4DF29
:10011000869508951F93CF93DF93F7DF182FAB9841
:100120008FE191E00197F1F700C00000C0E6D0E058
:10013000AA9A95E69A95F1F70000AA9880EC8A951C
:10014000F1F780E0BADFD8DF810F899390E0C736FE
:10015000D90771F7AB9A00000000CE010797DF9135
:10016000CF911F9108951F920F920FB60F921124F5
:100170008F939F93EF93FF9381B190E0887F883BAB
:100180009105C1F0893B91053CF4883A910559F0FD
:10019000803B910581F507C0803C910531F1883C99
:1001A000910549F522C081E080936F00809167003E
:1001B00083B915C080916F00863040F010926F00B7
:1001C00080916D0083B986B78F7B11C0E82FF0E076
:1001D000E959FF4F908193B98F5F80936F0086B785
:1001E000806486BF10926E0006C086B7806486BFAA
:1001F00081E080936E0086B7806886BFFF91EF91A3
:100200009F918F910F900FBE0F901F90189588238C
:1002100011F481E001C08E7F82B985E486BF089524
:10022000282F392FD901E7E6F0E08D91819380E006
:10023000EE36F807D1F710926E00089581E09091A4
:0E0240006E00992309F480E00895F894FFCF32
:0E024E00808080808080804242424242424254
:00000001FF
